S01D000062696E2F6F70656E626C745F73746D3332673037312E7372656394
S3150800000000900020AD030008FD030008FD0300086A
S3150800001000000000000000000000000000000000D2
S31508000020000000000000000000000000FD030008BA
S315080000300000000000000000FD030008851200080B
S31508000040FD030008FD030008FD030008FD03000882
S31508000050FD030008FD030008FD030008FD03000872
S31508000060FD030008FD030008FD030008FD03000862
S31508000070FD030008FD030008FD030008FD03000852
S31508000080FD030008FD030008FD030008FD03000842
S31508000090FD030008FD030008FD030008FD03000832
S315080000A0FD030008FD030008FD030008FD03000822
S311080000B0FD030008FD030008FD0300081E
S315080000BC10B5064C2378002B07D1054B002B02D024
S315080000CC044800E000BF0123237010BD380400204B
S315080000DC0000000004190008084B10B5002B03D0CB
S315080000EC0749084800E000BF07480368002B00D101
S315080000FC10BD064B002BFBD09847F9E70000000013
S3150800010C3C040020041900083804002000000000F4
S3150800011C002243088B4274D303098B425FD3030A2C
S3150800012C8B4244D3030B8B4228D3030C8B420DD33F
S3150800013CFF22090212BA030C8B4202D312120902CD
S3150800014C65D0030B8B4219D300E0090AC30B8B420B
S3150800015C01D3CB03C01A5241830B8B4201D38B03B9
S3150800016CC01A5241430B8B4201D34B03C01A52415E
S3150800017C030B8B4201D30B03C01A5241C30A8B42A1
S3150800018C01D3CB02C01A5241830A8B4201D38B028C
S3150800019CC01A5241430A8B4201D34B02C01A524130
S315080001AC030A8B4201D30B02C01A5241CDD2C309A2
S315080001BC8B4201D3CB01C01A524183098B4201D31E
S315080001CC8B01C01A524143098B4201D34B01C01A09
S315080001DC524103098B4201D30B01C01A5241C30881
S315080001EC8B4201D3CB00C01A524183088B4201D3F0
S315080001FC8B00C01A524143088B4201D34B00C01ADC
S3150800020C5241411A00D20146524110467047FFE747
S3150800021C01B5002000F006F802BDC0460029F7D04B
S3150800022C76E770477047C04670B50D4E0D4D0024E5
S3150800023CAD1BAD1005D0A300F35801349847A54261
S3150800024CF9D101F059FB084E084D0024AD1BAD1031
S3150800025C05D0A300F35801349847A542F9D170BDCF
S3150800026C5C1B00085C1B00085C1B0008641B000870
S3150800027C034B10B5002B02D0024800F005F810BD50
S3150800028C00000000A502000810B50100002300229A
S3150800029C002000F01BF810BD70B5094B094CE41A88
S315080002ACA41009D0084AA518AD00ED182B68013C16
S315080002BC9847043D002CF9D101F024FB70BDC046CB
S315080002CC641B0008681B0008FFFFFF3FF8B544468F
S315080002DC5F4656464D469B462F4BF0B41C68A423E6
S315080002EC5B000500E0580E00904600284BD043688A
S315080002FC1F2B0DDC5C1C002D21D102339B004460A6
S3150800030C1E5000203CBC90469946A246AB46F8BD0A
S3150800031C224B002B3CD0C820400000E000BF002830
S3150800032C36D0A42200235200A15843600160A05085
S3150800033C40328350043283500124002DDDD09A00BC
S3150800034C91468144424688214F467A50C42252002F
S3150800035C9046804442468739994012688A460A4331
S3150800036C9446424661461160842249465F465200CD
S3150800037C8F50022DC1D1020055468D32FF321168BD
S3150800038C0D431560B9E720004D30FF30E050AEE75D
S3150800039C01204042B6E7C0461C19000800000000C0
S315080003AC0D488546002103E00C4B5B58435004313D
S315080003BC0B480C4B42189A42F6D30B4A02E0002320
S315080003CC13600432094B9A42F9D300F013F8FFF77D
S315080003DC2BFF00F021FCFEE700900020681B0008AC
S315080003EC000000203804002038040020640900208E
S315080003FCFEE700008022024B12059A607047C04641
S3150800040C00ED00E0A0220300D205904217D0144A52
S3150800041C904218D0134A904219D0134A90421AD0D7
S3150800042C124A0120934200D070472021104B5A6A79
S3150800043C0A435A625A6A00208A435A62F4E70C4BFA
S3150800044C01215A6AF4E70A4B02215A6AF0E7084B6B
S3150800045C04215A6AECE7064B08215A6AE8E7C046B3
S3150800046C0004005000080050000C00500014005006
S3150800047C00100240F0B547460D6880B44A68002D56
S3150800048C24D0012300249C466346A3402B4019D054
S3150800049C1E005E437700BF19FF4372430568B846D2
S315080004AC3D40154305604A68551E012D2AD942461A
S315080004BC0F69C56877432A403A43C2604A68022ADC
S315080004CC11D00D682B000134E340DDD1013A012A25
S315080004DC05D84268CB68AA435D431543456000209E
S315080004EC04BC9046F0BDFF2B14D833007343026A44
S315080004FC1D01ED1AAA434D696B43134303624A68FF
S3150800050C0D68DFE747468D68826875433A402A438B
S3150800051C8260CCE71B0A5B435B43426A1D01ED1AFA
S3150800052CAA434D696B43134343624A68C9E7C046FD
S3150800053C70B5144C144B22680025134003432360F2
S3150800054C80239B00984201D0280070BD0F4B1049A0
S3150800055C1B685800C0184000FFF7DAFD8022666950
S3150800056CD200013023001100164202D1ECE7002814
S3150800057C05D05A6901380A42F9D10025E4E7032562
S3150800058CE2E7C04600700040FFF9FFFF2804002090
S3150800059C40420F00054B00205A69002A05DA044A26
S315080005AC9A60044A9A605869C00F70470020024046
S315080005BC23016745AB89EFCD8021044B09065A699F
S315080005CC0A435A615869C043C00F7047002002405D
S315080005DCF0B5474680B4050000F03EFE80268046FE
S315080005EC1C4FA844760201E06B1C19D13B69194CC7
S315080005FC3342F9D123691848802103401A00A369AC
S3150800060CC9050B40134311D0144A55682B43536044
S3150800061C20610120A3691943A16104BC9046F0BD71
S3150800062C00F01AFE8045E1D80320F6E700F014FE28
S3150800063C80262F18F60201E06B1C04D1236933427D
S3150800064CFAD10020E9E700F007FE8742F6D8032026
S3150800065CE3E7C04600200240FAC300005404002019
S3150800066CF0B5474680B4224E9846337807000D00FD
S3150800067C14000220012B02D104BC9046F0BD0123C4
S3150800068CFA203370002380007360FFF7A1FF00285F
S3150800069C23D1184A5369012F22D08021C9020B4352
S315080006AC5361EFF3108072B62200631CFF33291BCB
S315080006BC14688C5004329A42FAD180220D4952029F
S315080006CC0B691342FCD180F31088FA208000FFF7DF
S315080006DC7FFF084A5369BB43536100233370CBE74A
S315080006EC3B4353612C60BFF36F8F43466B60ECE75B
S315080006FC540400200020024010B50C4BDB68DB4389
S3150800070C9B0711D00A4B094AD068D16840044906A0
S3150800071CD468400E490F58430131FFF7F9FC610FB5
S3150800072C0131FFF7F5FC10BD024BECE70010024057
S3150800073C0024F40000127A00382110B50A4A93688E
S3150800074C0B40082B0DD0102B08D001211368074835
S3150800075C9B045B0F9940FFF7DBFC10BDFFF7CCFF42
S3150800076CFBE70348F9E7C046001002400024F400F2
S3150800077C00127A0070B50400FFF7DEFF1F220A4943
S3150800078C20608B68094D1B051B0F9B005B5913409A
S3150800079CD84060608B6806495B045B0F9B005B580E
S315080007AC1A40D040A06070BD001002402019000805
S315080007BC6019000810B50300032815D000200C2B6F
S315080007CC00D010BD224C626D1340C0221203134395
S315080007DC204A934236D0204A934228D01F4A934245
S315080007EC11D1FFF7A9FFECE7194C1D4A606D0340C0
S315080007FCC0208002034393421ED01A4A934216D055
S3150800080C194A9342EDD0FFF797FF1F21A268A368F8
S3150800081C1205120F154C920012595B040A40D0406F
S3150800082C5B0F134A9B009B581940C840C9E7E06DFB
S3150800083C8007C00FC003C4E7236800205B05C0D53A
S3150800084C0C48BEE723685B05BBD50A48B9E7C04622
S3150800085C0010024008000C000C000C0004000C00F0
S3150800086C020003000300030001000300201900081E
S3150800087C601900080024F400F0B557464E46454664
S3150800088CE0B4294E050033788A460220012B04D1A0
S3150800089C1CBC90469946A246F0BD0123FA2033703B
S315080008AC002380007360FFF793FE804600282CD146
S315080008BC2B68042B2DD0012352465B4213606C68BF
S315080008CCAB68E3189C421BD2184B194F994606E0A5
S315080008DCAA686B68944601346344A34210D94A4605
S315080008ECFA207B6980001340124A1343E200134333
S315080008FC7B61FFF76DFE0028EAD0534680461C60E4
S3150800090C02210B4A53698B435361002340463370CB
S3150800091CBEE7FA20064A0849536980000B4353611F
S3150800092CFFF756FE8046F0E75404002007FEFFFF4B
S3150800093C00200240020001000400010070B50368A3
S3150800094C040084B00D000120DB072AD42A698968C3
S3150800095C236811436A691143EA6911432E4A134005
S3150800096C0B43236062682D4B1340EA68134363609C
S3150800097CA2682B4B1340AA691343A360294B9C42CC
S3150800098C30D0294B9C4231D0284B9C420BD0284B5B
S3150800099C9C4208D001200F21E36A2A888B43134313
S315080009ACE36204B070BD01A8FFF7E4FE03980028C3
S315080009BCF0D06E68002EEDD080222B68E9691B04F6
S315080009CC1202DB0B914215D01A4A995AFFF7A0FB73
S315080009DC7308C0183100FFF79BFB0004000CE0609D
S315080009EC0020D8E70230FFF7E5FEE0E70C20FFF71A
S315080009FCE1FEDCE70F4A995AFFF78AFB73084000B9
S31508000A0CC0183100FFF784FB0B4B03400007400F5F
S31508000A1C1843E0600020BEE7F369FFEFFFCFFFFF46
S31508000A2CFFFCFFFF0038014000440040004800402E
S31508000A3C004C004080190008F0FF000070B5002833
S31508000A4C14DB032483082040FC342600134AC025F3
S31508000A5C9446C00089018640214081409B0063442E
S31508000A6CAD005A59B2431143595170BD03240F2393
S31508000A7CC0B203402040FC342500094AC000944605
S31508000A8C8901854021408140083B9B089B006344B3
S31508000A9CDA69AA431143D961E7E7C04600E100E0E9
S31508000AAC00ED00E00A4A431E012093420ED8C020EE
S31508000ABC084A094953600B6A00061B021B0A0343C2
S31508000ACC0B62002300209360073313607047C046FF
S31508000ADCFFFFFF0010E000E000ED00E0014B18609E
S31508000AEC7047C046280400200121002210B5074B88
S31508000AFC4942D962DA6219631A6399629A6259622F
S31508000B0C5A6200F05BF9002010BDC0460010024086
S31508000B1C10B50F4B04001968002901D1012010BD2E
S31508000B2CFA208000FFF7F4FA0A4B01001868FFF761
S31508000B3CEFFAFFF7B7FF0028F0D1032CEED80138EF
S31508000B4C00222100FFF77AFF034B00201C60E6E722
S31508000B5C30040020280400202C040020802110B525
S31508000B6C074A4900136803200B431360FFF7D0FFAD
S31508000B7C0123002802D100F0CBF80023180010BD81
S31508000B8C00200240014B18807047C0466E040020B6
S31508000B9C10B500F051FB0E4C236898420FD30D4B41
S31508000BAC1A78002A0CD000221A70A0232032DB05F2
S31508000BBC9A6200F041FB084B1B881818206010BD80
S31508000BCC01321A70A0231F32DB059A61F1E7C04681
S31508000BDC700400206C0400206E040020A023202240
S31508000BECDB059A627047C04610B5054B1B699B041A
S31508000BFC01D4002010BDFFF7F1FF0120FAE7C0462B
S31508000C0C0008005010B56420FFF7BCFF10BDC046A5
S31508000C1C10B5FFF7BDFF10BD10B5FFF79FFF80207D
S31508000C2C07248000FFF784FC2D4A1168A1430800AD
S31508000C3C02210143116013682340022B03D06D2156
S31508000C4C284800F0E3F88021274B49001A680A4324
S31508000C5C80211A601A00C9001068234B0842FBD081
S31508000C6CD968224A0A4022490A43DA60D968214AD5
S31508000C7C0A4021490A43DA60D968204A0A402049C1
S31508000C8C0A438021DA601A6849040A4380211A60EB
S31508000C9CDA6849050A438021DA6089041868124A19
S31508000CAC0842FBD00721936838208B43190002238E
S31508000CBC0B43936091680C4B01401029FAD1996843
S31508000CCC104A11480A409A609968104A0A409A6074
S31508000CDCFFF704FF00F0A6F800F0B2F8FCE7C046F0
S31508000CEC0020024098190008001002408C80FF1F53
S31508000CFC324000608C80C1FF324006008C80FFF1C8
S31508000D0C32400006FFF0FFFF0090D003FF8FFFFF75
S31508000D1CF0B50125274B8DB01A6C04202A431A64AA
S31508000D2C1A6CA0262A400592059A8022996B5200C5
S31508000D3C11439963996B00240A400492049A5A6BDE
S31508000D4C20272A435A635A6BF6052A400392039ABC
S31508000D5C596B014359635A6B02400292029A8022DC
S31508000D6CD96B92021143D963DB6B06A91A4001921F
S31508000D7C3000019B06970795089409940A94FFF787
S31508000D8C79FB8023B7629B0106A90B480693079447
S31508000D9C0A94FFF76FFB0C2306A9069330000A3B4F
S31508000DAC0793089409940A940B95FFF763FB0DB007
S31508000DBCF0BDC046001002400008005010B5A02433
S31508000DCC2023E405A3620D48FFF71CFB2000FFF760
S31508000DDC19FB0B4B0B4AD96B0A400421DA635A6B85
S31508000DEC8A435A635A6B03398A435A63986B064A81
S31508000DFC02409A631A6C8A431A6410BD00080050A4
S31508000E0C00100240FFFFFDFFFFFEFFFF10B500F0CC
S31508000E1C05F8FCE710B5FFF7F5FE10BD10B5FFF7A2
S31508000E2CF7FE10BD10B500F071FCFFF7F3FF00F0EC
S31508000E3CDDF900F0A3FC00F03DF800F02BF810BD2E
S31508000E4C10B5FFF7EBFF00F0E9F900F03FF800F0FA
S31508000E5C01F810BD10B500F073F8012803D00A4C40
S31508000E6C2378012B00D010BD00F0E6F9074B1A6861
S31508000E7C074B1B68D318F533FF339842F3D300237B
S31508000E8C237000F047FCEEE7780400207404002079
S31508000E9C7C0400200122054B10B51A7000F0CCF921
S31508000EAC034B1860FFF7D6FF10BDC0467804002028
S31508000EBC7C04002010B500F04BF800F091FC0022E1
S31508000ECC014B1A7010BDC0463404002010B582B010
S31508000EDC6B46094CD91D200000F0BEFC012801D038
S31508000EEC02B010BD0022054B20001A706B46D9794A
S31508000EFC00F04CF8F4E7C0468004002034040020C7
S31508000F0C7047C04610B5054B1B78002B02D1C9B2E9
S31508000F1C00F082FC00F032F810BDC0463404002004
S31508000F2C044B187802230138C0B2834280414042F0
S31508000F3C800170473404002010B5FFF7F1FF10BD8F
S31508000F4C10B500F013F8431E9841C0B210BDC04648
S31508000F5C00224321044B44205A5400211A709A64E7
S31508000F6C1A52997059707047C0040020024B1878B1
S31508000F7C431E9841C0B27047C00400200021432389
S31508000F8C014AD1547047C046C0040020F8B503780E
S31508000F9C0500934CFF2B0CD02278012A00D0F8BD03
S31508000FAC3733DBB2352B00D9FFE08E4A9B00D3587A
S31508000FBC9F4600220125E370EF3B62702371627134
S31508000FCC2570FFF7B9FFA071FFF7AAFFE071FFF7CD
S31508000FDCA7FF08224423000A20726572A572E25202
S31508000FEC00F0CCFB4323E35C012B05D04423E15EE4
S31508000FFC0029D4DD89B207E0FE2302220221E37020
S3150800100CEE3B23713433E25201224323E01CE254B3
S3150800101CFFF778FFC3E7FFF78FFF6B780138984225
S3150800102C5CDDFF230122E370BB3BE25269780029A1
S3150800103C00D0C7E000F0B6FB0028D3D1FE2302226D
S3150800104CE370CD3B23711333E2524323E35C012B4C
S3150800105CD2D04423E15AD7E700F05CFBFF230122E8
S3150800106CE370BB3BE252F0E74168A06C00F08EFBE4
S3150800107C0028F3D1E2E70025FF232571E37065719B
S3150800108CFFF75AFF07224423A071E5712572657292
S3150800109CE252DAE7FF23E3704668A76C0025002EB8
S315080010AC08D03B78013EED18EDB20137FFF7B6FED6
S315080010BC002EF6D1002201230021E57123712D0E95
S315080010CC6271A2714333083221726172A572E252BF
S315080010DCBBE7FFF731FF6B7898426EDCFE230222E2
S315080010ECE370DC3B23712233E252AEE7FE23E37056
S315080010FC0023022223714433E252A6E7FF236278C7
S3150800110CE3700023627106222371A371E3712372C3
S3150800111C4433E25299E70023237063709EE7A66C6A
S3150800112CFFF70AFF6A1C411E300000F02BFB002853
S3150800113C84D0FF23E370FFF7FFFEA36C01229C46C5
S3150800114C442301386044A064E2527EE7FF23E3702F
S3150800115C43680122A3644423E25276E7FF23E37033
S3150800116C214B0721A3640023082223716371A37101
S3150800117C23726372A3724433E171E25265E7FFF797
S3150800118CDBFE6A789042A9DDA16C92B2201D00F0B4
S3150800119CE3FAFF23A26CE370944644226B7863440B
S315080011ACA3646B780133A3521CE7FE230222E37077
S315080011BCDE3B23712433E25247E76968201DA1649C
S315080011CC6A78E4E7AA1CA06C00F0DCFA002800D1C7
S315080011DC34E7A26C6B7894466344A36402E7C04672
S315080011ECC0040020A0190008781A00080022054B34
S315080011FC05491A60596005219A601960034B1A60F3
S3150800120C7047C04610E000E0FFF900000C0500200E
S3150800121C0022014B1A60704710E000E0044B1B6873
S3150800122CDB0303D5034A1368013313607047C046C2
S3150800123C10E000E00C050020054B1B68DB0302D40C
S3150800124C044B18687047034B1A68501C1860F9E76A
S3150800125C10E000E00C050020054B1B68DB0302D4EC
S3150800126C044B18687047034B1A68501C1860F9E74A
S3150800127C10E000E00C0500207047C046F0B5474664
S3150800128C0F4B80B4984607001C0000250D4E00E055
S3150800129C2668FFF7C3FDBE4204D863689C466644BD
S315080012ACB74207D301350C340F2DF1D1FF2004BCFE
S315080012BC9046F0BD6B005D19AD004544287AF6E7FB
S315080012CC801A000800200008F0B5454657464E46D9
S315080012DCE0B480460068FFF7D1FFFF282CD0FFF753
S315080012EC59F943461C1D81239B0043449A46042303
S315080012FC42465B429B1A994608E02A686B689642F6
S3150800130C16D19F4214D1083454451CD026686768F8
S3150800131C4B461D1943461B689C466544FFF77EFDE4
S3150800132C32003B0029000120FFF79AF90028E4D087
S3150800133C0024FFF741F900E0002420001CBC90466D
S3150800134C9946A246F0BD0124F3E7C046114B70B589
S3150800135C04000D0098421BD00F4A914205D0FFF7A6
S3150800136CB3FF01280ED000240AE01C002368AB4208
S3150800137C06D02000802220C09200290000F0ECF94B
S3150800138C200070BD002CEED0EB05EFD00024F7E75B
S3150800139C024CF9E71005002000200008140700206D
S315080013ACF0B54E4657464546E0B41E004B0A5B025E
S315080013BC9946036807000C0015005A1C38D0994545
S315080013CC06D038004946FFF7C1FF071E2ED0036822
S315080013DCE41A3B1D98461C4B3C199A4601339C460D
S315080013EC0434E14406E02B78013E237001350134C0
S315080013FC002E15D0FFF712FD4346E31A5345F2D9D2
S3150800140C38004946FFF7A2FF071E0FD0031D1C0024
S3150800141C98462B78013E237001350134002EE9D10C
S3150800142C01201CBC90469946A246F0BD0020F8E760
S3150800143C03004A4604C3802218009200494600F06D
S3150800144C8BF93B68BBE7C046FF0100000123034A42
S3150800145C5B421360024A13607047C04614070020AB
S3150800146C1005002010B5FFF7F1FF10BD134B70B532
S3150800147C16004A1E04000D001B1A9A4201D90020B8
S3150800148C70BDFFF7FBFEFF28F9D0601E4019FFF769
S3150800149CF5FEFF28F3D00A4A630A5B02934206D08C
S315080014AC2B00320021000748FFF77AFFE8E72B00EC
S315080014BC320021000448FFF773FFE1E7FFFF01083C
S315080014CC002000081407002010050020F0B54D4632
S315080014DC44465F465646F0B44F4B4A1E87B0040046
S315080014EC0D001B1A9A4273D8FFF7C8FE013C070079
S315080014FC6019FFF7C3FE0600FF2F69D0FF2E67D0D1
S3150800150C002300240293B74263D8032F61D91C0029
S3150800151C122E5ED8414B0025994698461C0004238A
S3150800152C9A4601E0237A9A46FFF778FCBA4566D0C4
S3150800153C0135EDB20C340F2DF4D1394B9B460123F2
S3150800154C5B429A4647460424002500E03C7AFFF79E
S3150800155C65FCA6424DD00135EDB20C370F2DF5D1F1
S3150800156C01277F420425002401E043461D7AFFF734
S3150800157C55FCAE4237D00C239C460134E4B2E04409
S3150800158C0F2CF2D100235246BD1AED1802230393F1
S3150800159C5B4604930123ED0AADB205930024FEF7CE
S315080015ACF9FF002D08D11CE0049B01340193A4B269
S315080015BC01330493A54214D9FFF730FC02A903A8FA
S315080015CCFFF75AF90028EFD00024FEF7F5FF00E0E4
S315080015DC0024200007B03CBC90469946A246AB4670
S315080015ECF0BD0124F1E763001C19A4004C446368A0
S315080015FCC9E76B005D194B46AD005F59B2E76B0046
S3150800160C5D194B46AD005B59F8279A463F06574479
S3150800161CFB0A9B4696E7C046FFFF0108801A00089E
S3150800162CFFFF1E0000B5114B83B01A68012001326A
S3150800163C19D098685A68844662441100DA680C48CE
S3150800164C94461A69614494465A69614494469A695F
S3150800165C61449446DA6961448B185B4201AA0421F9
S3150800166C0193FFF703FF03B000BDC0461005002029
S3150800167CBC2000080D4B18680D4B1B68C0180D4B89
S3150800168C1B68C0180C4B1B68C0180C4B1B68C01881
S3150800169C0B4B1B68C0180B4B1B68C0180A4B1B68F6
S315080016ACC01843425841C0B27047C04600200008D3
S315080016BC04200008082000080C2000081020000848
S315080016CC1420000818200008BC20000810B50B4888
S315080016DC0368013306D0FFF7F7FD03000020002B43
S315080016EC00D110BD06480368013305D0FFF7ECFDA1
S315080016FC431E9841C0B2F4E70120F2E7100500201A
S3150800170C14070020004870470020000810B500F0A8
S3150800171CEFF810BD10B500F03DF8002800D110BD4B
S3150800172CFFF762FA0028FAD0FFF7EAFBFFF770FD1D
S3150800173CFFF7DAF900F032F8054B1840054B9860BC
S3150800174C00F02CF8446800F0D5F8A047E7E7C04647
S3150800175C80FFFF1F00ED00E070B5551EADB2002AE4
S3150800176C0AD00C006D180135461A23783355013406
S3150800177CFFF754FBAC42F8D170BDC04610B5FFF765
S3150800178C71FE10BD10B5FFF771FE10BD10B5FFF751
S3150800179C9DFE10BD10B5FFF76DFF10BD10B5FFF718
S315080017ACB1FF10BD10B5FFF73DFF002801D0FFF7BC
S315080017BC8DFF10BD70B5094C8026A062FFF73CFD65
S315080017CC0A30050005E0FFF729FBFFF735FD8542D2
S315080017DC02D3E3691E42F6D070BDC04600440040F1
S315080017ECE12310B51B0288B001930C220023094C87
S315080017FC6946200002930393049305920693079374
S3150800180C0093FFF79BF8012322681343236008B063
S3150800181C10BDC0460044004070B504000D004029B8
S3150800182C12D82800ADB2FFF7C5FF002D0BD0013D2D
S3150800183CADB201356519FFF7F1FA20780134FFF7D7
S3150800184CB9FFAC42F7D170BD74210248FFF7DEFA36
S3150800185CE7E7C046341B0008F8B5204D0E002C7877
S3150800186C002C06D11E4BDA69920626D400242000D9
S3150800187CF8BD20241A4AD3691C4015D0194C1A49AC
S3150800188C2378576ACA18577001330A78DBB2237063
S3150800189C9A42EBD192B20131FFF75EFF00232B700F
S315080018AC237801243370E2E7FFF7C6FC0F4B1B685D
S315080018BC64339842DAD92C70D8E75B6A0A4ADBB2E9
S315080018CC1370013B3F2BD1D8FFF7B6FC074B1860BA
S315080018DC044B1C7001232B70C9E7C046190900205C
S315080018EC0044004018090020200900201C0900208B
S315080018FC72B6704762B67047F8B5C046F8BC08BCF5
S3150800190C9E467047F8B5C046F8BC08BC9E4670475C
S3150800191C000000200000000000000000000000008D
S3150800192C000000000000000000000000000000009D
S3150800193C0000000001000000020000000300000087
S3150800194C0400000006000000070000000800000064
S3150800195C0900000000000000000000000000000064
S3150800196C0000000001000000020000000300000057
S3150800197C04000000010002000400060008000A002A
S3150800198C0C00100020004000800000016D61696E9B
S3150800199C2E6300002A110008B6110008B6110008BB
S315080019AC48100008B6110008B611000864100008A3
S315080019BC221000087410000882100008B6110008DE
S315080019CCB6110008B6110008B6110008B6110008C1
S315080019DCB6110008B6110008B6110008B6110008B1
S315080019ECB6110008B6110008B6110008B6110008A1
S315080019FCB6110008B6110008B6110008B611000891
S31508001A0CB6110008B6110008B6110008B611000880
S31508001A1CB6110008B6110008B6110008B611000870
S31508001A2CB6110008B6110008B6110008B611000860
S31508001A3CB6110008B6110008B6110008A010000867
S31508001A4CDE1000088A11000858110008B6110008A3
S31508001A5CB6110008B611000868110008B61100087E
S31508001A6CF810000808110008221100084F70656E5E
S31508001A7C424C540000200008000800000400000036
S31508001A8C00280008000800000500000000300008C7
S31508001A9C00080000060000000038000800080000D6
S31508001AAC07000000004000080008000008000000BD
S31508001ABC0048000800080000090000000050000853
S31508001ACC000800000A000000005800080008000082
S31508001ADC0B00000000600008000800000C00000065
S31508001AEC00680008000800000D00000000700008DF
S31508001AFC000800000E00000000780008000800002E
S31508001B0C0F00000000800008008000001000000094
S31508001B1C0000010800800000110000000080010888
S31508001B2C00800000120000002E2E2F2E2E2F2E2E97
S31508001B3C2F536F757263652F41524D434D305F536A
S31508001B4C544D333247302F756172742E6300000082
S30D08001B5C7D020008E5000008FF
S30908001B64BD000008AA
S31508001B6800000000EC02002054030020BC030020FB
S31508001B78000000000000000000000000000000004F
S31508001B88000000000000000000000000000000003F
S31508001B98000000000000000000000000000000002F
S31508001BA8000000000000000000000000000000001F
S31508001BB8000000000000000000000000000000000F
S31508001BC800000000000000000000000000000000FF
S31508001BD800000000000000000000000000000000EF
S31508001BE800000000000000000000000000000000DF
S31508001BF800000000000000000000000000000000CF
S31508001C0800000000000000000100000000000000BD
S31508001C180E33CDAB34126DE6ECDE05000B00000082
S31508001C28000000000000000000000000000000009E
S31508001C38000000000000000000000000000000008E
S31508001C48000000000000000000000000000000007E
S31508001C58000000000000000000000000000000006E
S31508001F8800000000000000000024F400040000001F
S30D08001F9801000000040000002E
S705080003AD42
